:1000000000308A003A280000831A0A28A500030E4F
:10001000A6000F288312A500030EA600A6140A0846
:10002000AD008A018313A50E0408A7002008A800CC
:100030002108A9002208AA002308AB002408AC006C
:1000400083128B1E25280B194028270884002808B6
:10005000A0002908A1002A08A2002B08A3002C0850
:10006000A4002D088A00260E83008312250EA618F0
:1000700083160900FF2383168F0000308A00A02812
:100080003508BF000930A000A00B44280000000084
:100090001F151F1949281E08B50035083F02031C0B
:1000A000552835083F02C00058283F083502C000D7
:1000B0004008013C031C5F280130B6076028B601E8
:1000C0003608063C031867283508B400B6010B1142
:1000D0008A1125283E308400000803197E2801304B
:1000E000A100A001A00B7228A10B71284A30A0002A
:1000F000A00B782800000000800B6F280034BB01A3
:1001000039083B020318982805156430BE006A20A0
:10011000BC013A083C0203189228C830BE006A208D
:10012000BC0A89280511C830BE006A20BB0A802895
:100130000430BD00FA30BE006A20BD0B9A2800349E
:1001400084011F30830583161F149F141F1583120B
:10015000AE010130AF00B001B101B20183161F1032
:100160009F141F150B30650083121F139F171F1458
:100170000730A000A01DC428073081018130840011
:100180000008C0390F388000640081308400000806
:10019000C039200480000030A1001F08C7392104A5
:1001A0009F008B16B501B401B601C0308B048501E8
:1001B00085160430B900FA30BE006A20B90BDB287E
:1001C000B630B3003408A43C031CEE28B301083059
:1001D000B9000230BA007F208516FF283408E93CB8
:1001E000031CF8280330B9000230BA007F20FF2832
:1001F000B3010830B9000230BA007F208516043000
:10020000B900FA30BE006A20B90B0129B3080319FE
:1002100021293408A43C031C15290830B9000230F8
:10022000BA007F208516B301202933083402031851
:100230001F290130B900BA007F20851620298512B8
:040240000629630028
:02400E00643F0D
:00000001FF
